:020000040800F2
:1000000000020020A50400081105000821050008D1
:10001000E9060008F90600080907000800000000CA
:100020000000000000000000000000004104000883
:100030001907000800000000250400080B02000852
:100040000B0200080B0200080B0200080B0200085C
:100050000B0200080B020008E9130008E91300086E
:10006000E9130008E9130008E91300080B0200086F
:100070000B0200080B020008091200080B0200081E
:100080000B020008DD1100080B0200080B0200083B
:100090000B0200080B0200080B020008E91300081D
:1000A0000B0200080B0200080B0200080B020008FC
:1000B000451600080B0200080B0200080B0200089E
:1000C0000B0200080B0200080B020008413A00086E
:1000D0004D3A00080B020008D1110008FD1100087C
:1000E000E91300080B0200080B0200080B020008CD
:1000F0000B0200080B0200080B0200080B020008AC
:100100000B0200080B020008511600080B02000841
:100110000B0200080B0200080B0200080B0200088B
:100120000B0200080B0200080B0200080B0200087B
:100130000B0200080B0200080B0200080B0200086B
:100140000B0200080B0200080B0200080B0200085B
:100150000B0200080B0200080B0200080B0200084B
:100160000B0200080B0200080B0200080B0200083B
:100170000B0200080B0200080B0200080B0200082B
:100180000B0200080B02000800F0D6BA704700000E
:1001900070B50C46064600F073F9094B094A1D6814
:1001A0002C44944202D8084A944207D20C2333606C
:1001B0004FF0FF3500F06CF9284670BD1C60F9E780
:1001C0000002002000000220D4130020194610462F
:1001D00000F0BEBA1946104600F0C2BA13230360FD
:1001E0004FF0FF307047132303604FF0FF3070472C
:1001F000132303604FF0FF30704702294FF00003D4
:1002000003608CBF00200120704700F08DBA000011
:10021000114B70B500241C60104B114D18682E68EE
:1002200000F09CF80F4B53F820301B68A3F1080234
:1002300096420FD026B13179092904BF0A213171C4
:10024000092103F8041C33F9021C074B2A601980AA
:10025000012070BD204670BD2C0400202004002029
:10026000280400203404002024040020082930B58C
:1002700003791AD9082B14D842791A4B53F8225013
:1002800000F108047DB12D68856053F822502C6080
:1002900043F82240144A44790123A34014682343BD
:1002A0001360017130BD8460F2E7082BF9D94579FC
:1002B0000C4B53F825203AB11468A2420BBF002220
:1002C000246843F825201460427953F82230002B2B
:1002D000E7D1054C012303FA02F2236823EA020363
:1002E0002360DEE7340400202004002008B50A4B18
:1002F0001B681A79082A02D95B7983420AD900F06F
:10030000CAF818B1054B01221A6008BDBDE80840C3
:1003100000F080B808BD00BF280400202C04002095
:1003200008B500F0ADF8094B094A1B88094D1BB20E
:10033000002442F82340084A286813682146013BFC
:100340001360FFF793FF2C6000F060F82404002096
:100350007404002028040020300400200023C20779
:1003600001D51846704740080133F8E7134423F0DD
:10037000030310B54FF077321C1F43F8042C6207BB
:1003800042BF4FF0883243F8082CA3F108044FF025
:10039000807304E909000F4B44F80C3C002344F837
:1003A000103C032344F8143C2246022344F8183C32
:1003B000012344F81C3C42F8201D0B2342F8043D65
:1003C000013B032BFAD120466FF0020340F8443D75
:1003D00010BD00BF210300080548064A064B01680E
:1003E000914201D1984201D3181A70470430F6E7C0
:1003F00000000020FEE7FEE700020020EFF3088087
:1004000070470000004870470000002000F03CF8F2
:1004100001DFFEE7024A536843F0805353607047A0
:1004200000ED00E0EFF3098020E9F00F40F804ED63
:1004300002490968086000F003F800002804002061
:10044000FFF7E6FE04480068016801C9B1E8F00F53
:1004500081F309880047000028040020BFF34F8F74
:100460000549064BCA6802F4E0621343CB60BFF350
:100470004F8F00BFFDE700BF00ED00E00400FA056C
:10048000EFF3108072B6704762B6EFF310807047DA
:1004900080F310887047EFF30580C0B27047704753
:1004A0007047000008B5FFF7FAFF6A46114B124982
:1004B000934213D3114A124B12498B4211D3124B60
:1004C000124A0021934211D3FFF7EAFF00F022FB0A
:1004D00004F0DEF8BDE8084000F076BB43F8041BEA
:1004E000E6E752F8040F43F8040BE6E743F8041B71
:1004F000E8E700BF00000020FEE7FEE7C465000853
:10050000000200202004002020040020D41300203A
:1005100008B50249042000F01BFB00BF7B5B00080C
:100520000D490E4A0E4B6846904203D8984201D9B5
:10053000002102E009468D46012104207246024254
:1005400002D1EFF3088001E0EFF309802DE9F00F0D
:100550006B4600F007F800BF0002002000000220F8
:10056000600500202DE9F04F9A46494B8FB0934625
:100570009A6B03925A6B04929F6ADA6A05921A6B1D
:10058000DB6B0793434B06921A68434B9A4204462F
:10059000884602D0414804F0E1F9B8F1000F4ED08E
:1005A0003F4804F0DBF900252E463E4804F0D6F91A
:1005B00039463D4804F05EF905993C4804F05AF983
:1005C00006993B4804F056F907993A4804F052F965
:1005D0003A0403D50399384804F04CF93B0603D597
:1005E0000499364804F046F9354804F0B7F95946FD
:1005F000344804F03FF9B8F1000F1BD1324804F041
:10060000ADF93146314804F035F96946304BC91A25
:1006100003D549422F4804F02DF920468268C3686B
:1006200001698C4641698E46AD46514691E8F00F0E
:100630004168006801BE2849052000F089FA94E865
:100640000E00E068D4F81C90089020690990606959
:100650000A9019F4007F2148A6690D930CBF04F19C
:10066000200504F124050C920B9104F077F9089B06
:1006700000930BA90EC91A4804F0FCF8CDF80090BD
:1006800033460A9A0999174804F0F4F88DE700BF39
:1006900000ED00E000000020FEE7FEE774590008CE
:1006A0008A5900084F5A0008585A0008685A00082A
:1006B000785A0008885A0008985A0008A85A000872
:1006C000B85A0008BD5A0008CF5A0008005B00085D
:1006D00058010020285B0008555B0008B959000844
:1006E000D4590008115A000808B50249062000F044
:1006F0002FFA00BF685B000808B50249072000F028
:1007000027FA00BF4259000808B50249082000F046
:100710001FFA00BF875B000808B50249092000F0F6
:1007200017FA00BF5459000808B502490A2000F022
:100730000FFA00BF66590008034B044A4FF4E13139
:10074000002000F07FBC00BF04020020110F000851
:100750000A460146014800F0E6BB00BF0402002043
:1007600010B50A460C460146002000F015FC204654
:1007700010BD002000F0EEBE034B1968024611B90F
:10078000084600F0AFBE70473805002010B5094A92
:10079000136843B19C6881688C4207D303D15C68BD
:1007A00041688C4202D90360106010BD1A461B6874
:1007B000EFE700BF40050020F0B51F4E1F4D336826
:1007C0001F4C013333601F4B00201A6818602B68E0
:1007D000226019460746B64621B1DEF800C08E6891
:1007E000664503D900B1296027B9F0BD0F46012045
:1007F0000968F1E700213960DAB163B151685868DE
:10080000814294BF11461946084612681B6822B9F6
:1008100003602160F0BD1146F6E70BB90260F8E70E
:1008200055685E68B54294BF15461D46056028466A
:10083000EBE72360F0BD00BF3C0500204005002031
:1008400048050020440500202DE9F0412C4F2D4C97
:1008500001233B60236893B9FFF7AEFFFFF789FFE1
:100860000130FBD000254FF0000823685BB9FFF78B
:1008700080FF854224D9FFF79FFF0025F5E7FFF7AA
:1008800078FF0546EFE75E68FFF773FF854204D8FF
:10089000864202D9361A132EE9D823685E68FFF71C
:1008A00068FF854201D88642F7D823681A6822601B
:1008B000C3F80480C3F80880DA6818699047D4E761
:1008C00023686BB15E68FFF754FF063E1430864222
:1008D000CBD300233B603046BDE8F041FFF74CBF6F
:1008E000FFF747FF85420646C5D810F1140F04D321
:1008F000FFF73FFF8642FBD9BDE74FF0FF36E8E741
:100900003805002048050020144B1A6882420FD198
:1009100012681A601AB150680638FFF72DBF4FF001
:10092000FF30FAE7904202D102681A60704713461E
:100930001A68002AF6D10A4A13681BB9094A1368D3
:100940003BB97047984202D10368136070471A465A
:10095000F2E79842F8D01A46F1E700BF48050020B8
:10096000440500204005002008B500231846054A2C
:10097000054900F01DFE4FF0FF30BDE80840FFF7CD
:10098000FBBE00BF4908000840420F00F8B504460E
:100990000D46FFF7EEFE002385420646236011D385
:1009A000A5F10A0383420DD20A35FFF7E2FE854224
:1009B000FBD3FFF7DEFE8542FBD8E368206998474A
:1009C0000020F8BDFFF75CFD63680746002B33D1BC
:1009D000A368002B30D11A4B65601A681B68B542BA
:1009E00038BF0132A260A2689A4206D92046FFF7BA
:1009F000CDFE3846FFF74CFDE2E7B5420FD9114B6B
:100A000019461A6812B15068854213D222601C60E0
:100A10000B689C42EDD1A81FFFF7AEFEE9E70A4A3A
:100A2000136813B159688D4202D223601460E0E765
:100A30001A46F5E71346E4E72046FFF765FFCAE7E5
:100A40003C050020480500204405002038B5044638
:100A5000FFF716FD6368054633B9A36823B9284636
:100A6000BDE83840FFF714BD2046FFF74DFFF6E71D
:100A7000C36870B504460D46C3B1FFF7E7FF092D03
:100A80000CD8FFF776FE0646FFF773FE801B854203
:100A9000FAD8E3682069BDE870401847FFF769FE9F
:100AA00029182046BDE87040FFF770BF70BD0000F8
:100AB0002DE9F04704460E4690461AB9BDE8F047C6
:100AC000FFF7D6BFFFF7DCFC63680746E3B9A3680E
:100AD000D3B9DFF83CA0FFF74CFEDAF800508146AE
:100AE000FFF747FE8145F6D8304408EB0502864201
:100AF00088BF01326060A2602046FFF747FE38469B
:100B0000BDE8F047FFF7C4BC2046FFF7FDFEE0E775
:100B10003C05002008B50121094800F085FB0121B2
:100B2000084800F081FB0121074800F07DFB01210E
:100B3000064800F079FBBDE8084000F033B900BF7B
:100B40000D0C02400C0C02400E0C02400F0C024037
:100B500008B50E4B1A680C469AB9012203281A6090
:100B600003D171460A4803F085FE2146094803F087
:100B700081FE00F073FD084803F07CFE074803F097
:100B800079FEFFF77DFC00F0FBF800BF4C0500206C
:100B9000AD5B0008B15B0008D95B0008CD5B0008C5
:100BA00008B5034803F066FE00F050FE002008BDC3
:100BB000DB5B000808B5034C2368012000F072F9E4
:100BC000FAE700BF500600201FB5FFF759FC0E4B97
:100BD0000E481B68029300240D4B00930F220C2338
:100BE0004FF48071019400F055F80A4B0A481B68D5
:100BF00002930A4B009307220C234FF4C061019427
:100C000000F048F8FFF702FC180200205005002011
:100C1000B50B00081C02002054060020A10B0008A0
:100C200008B5FFF72DFC094B1B681A79082A07D96C
:100C30005A79074B53F8221011B1096843F8221072
:100C4000FFF726FCBDE80840FFF7E4BB28040020BE
:100C50003404002038B50B79082B03D90849032048
:100C6000FFF776FF4C7901F10802036813B98B6036
:100C7000026038BD13F8035CAC42F8D31846F4E7C1
:100C80009B5B0008031F53F8042F9A42FBD0181AED
:100C9000704700000F2A2DE9F74F05468B46914615
:100CA0009A4633D810F003031BBFC3F10403ED18B9
:100CB0000B46CB1A303B23F003031AF0080F05EB69
:100CC000030419D02A46A24213D30193FFF7D8FB9D
:100CD0002949019B8046012251F8226017B2C6B112
:100CE0000132212AF8D14046FFF7D2FB6FF08A0784
:100CF0003DE012600432E6E72D60E6E70121204680
:100D0000FFF7B4FA4046FFF7C3FB30E06FF015077A
:100D10002DE041F822400C98E7802A460D99FFF714
:100D200025FB0E9B154AA3624FF0FF33E361136866
:100D3000206001331AF0010F6562C4F82CB084F80A
:100D400005902671A660E66026616661A66126624E
:100D50001360D3D10A212046FFF788FA1AF0040F56
:100D6000D0D14046FFF794FB4846FFF7BFFA38461C
:100D700003B0BDE8F08F00BF7404002030040020F1
:100D800008B5EFF30581C1F3080119B11039044822
:100D900003F070FD00BE042000F084F8FBE700BF04
:100DA000285C000810B53C4C02F0E6F80022A26076
:100DB000236823F0867323F480332360E260236882
:100DC00043F48033236023689803FCD54FF08051AF
:100DD000002000F0B7FC314A136843F4004313606D
:100DE000A36823F0F003A360A368A360A36823F4BF
:100DF0006043A360A36843F40043A360A36823F4A3
:100E0000E053A360A36843F4A053A360002363608E
:100E1000636843F480036360636843F008036360BE
:100E2000636843F4A843636063686360636843F086
:100E3000E0636360236843F08073236002F5E4326B
:100E400013689901FCD5164B00211960196841F40B
:100E500000711960196841F480611960196821F006
:100E60000F011960196841F005011960936823F0BA
:100E700003039360936843F002039360064B1946A3
:100E80009A681207FCD51A6822F001021A600B68F2
:100E90009B07FCD410BD00BF00380240007000402A
:100EA000003C0240174B93F90010042806D8DFE8F5
:100EB00000F00307101C1C0000221A70084670473F
:100EC00001221A70104A136923F00403136130BF22
:100ED000F4E702221A700D4A136823F0030313602B
:100EE000094A136943F00403F0E703221A70074B21
:100EF0001A6842F00E021A605A6842F480725A6010
:100F0000EEE700BF2002002000ED00E0007000408E
:100F100038B50446043000F04EFC0546204601F08A
:100F2000C1FE284638BDF8B504460E461746051DD5
:100F30003A463146284600F029FC00B1F8BD0121AF
:100F4000204601F07FFEF3E74209012300F01F0075
:100F500003FA00F0014B43F82200704700E100E083
:100F6000024B1B680BB1FFF75BBE70472C040020DF
:100F700008B50B689B0608D5064B496803EBC00211
:100F8000C9B253F8303050689847BDE80840FFF7C1
:100F9000E7BF00BF640C00202DE9F84306460C466D
:100FA0001546FFF778FADFF8849078B118235E438E
:100FB000254459F80630AC4201D1BDE8F8831A68DF
:100FC0001206FCD514F8012B5A60F4E7134F4FEAD0
:100FD000860847440121384601F034FE182303FBFC
:100FE00006960F48F17C0F4A0729D8BF024601F048
:100FF0000701102013FB0103D118ADB2CC604D6086
:10100000D158094841F00101D1504044012101F07B
:1010100019FE3846BDE8F84301F044BE5C0C0020E0
:101020000060024000640240540C0020385C00085C
:10103000034A182303FB00204168407C00F082BB78
:10104000385C000801282DE9F84F05460C4600F2EF
:10105000A78018214143544F07EB01087E5853499C
:1010600041F8302001EBC0014FF000094B60504BBC
:1010700043F820904F48012140F8259000EB85006F
:1010800001F0E0FDD8F808B04946584600F0CCF829
:10109000D8F80C900121484600F0C6F898F810A046
:1010A0005846514600F066F95146484600F062F94C
:1010B0002846FFF7BDFF98F811302401002B4FD1CF
:1010C0003D48B0FBF4F002F06DFF804603F012F9EA
:1010D00084B2204602F06AFF0146404602F0B0FEAC
:1010E0004FF0834102F0B6FF03F004F9240100F051
:1010F0000F00A4B204438023B46073610023336102
:1011000042F20C03F360182303FB0573DC7C072C0D
:1011100028DC4FF40011022000F014FB274A1820AD
:10112000102104F0070310FB031300FB0570244992
:10113000057D90F9120002EB030E41EA4561D150A2
:10114000331DCEF808300023CEF81430FFF7FCFE34
:10115000062C0EDC04F10B0040B2FFF7F5FE0EE0AA
:101160001848AEE74FF48001022000F0EBFA164A6F
:10117000D5E7072C0AD1154B4FF400425A60F368AB
:1011800043F02003F3600020BDE8F88F0C2C02DC54
:1011900004F13000E0E70F2CF1DC04F13700DBE76D
:1011A0004FF0FF30BDE8F88F385C0008640C002079
:1011B0005C0C0020540C002080DE800200600240A5
:1011C0005004010000BD01050064024000E100E0A0
:1011D00001490020FFF7CCBE0044004008B5054B94
:1011E00005484FF40012DA6001F05CFDBDE80840EC
:1011F000FFF7B6BE00600240540C002001490120F8
:10120000FFF7B6BE0048004008B5054B05484FF053
:1012100000629A6001F046FDBDE80840FFF7A0BEFD
:1012200000600240580C0020F8B50D460126C0F3BE
:10123000832120F00F0400F00F0706FA01F10220CD
:1012400000F080FA07FA06FE0323226803FA0EF381
:10125000D84302402260226805F0030101FA0EF132
:1012600011432160E2681040E060E168C5F381024B
:1012700002FA0EF20A43E2606268BE4022EA060207
:1012800062606268C5F30015BD4015436560A268E1
:10129000B6B21343A36000206683F8BD2DE9F04188
:1012A00000F00F041746304A42F8343002EBC40213
:1012B000069B536005468846C0F383264FF4804161
:1012C000012000F03FFA41462846FFF7ADFF042C0D
:1012D000264B28DCA11D01228A401A60012F244BD5
:1012E0002AD032D3022F3AD004F00C0303F180430A
:1012F00003F59C3305F003059A68AD000F21A94062
:1013000022EA01029A609A6806FA05F515439D6083
:10131000012303FA04F4164B5C611A6814431C6041
:101320000020BDE8F081092C02DC4FF40002D4E774
:101330004FF480725A60D1E79A68A7403A439A60A6
:10134000DA6822EA0707DF60CEE799680122A24047
:1013500021EA02019960D9680A43DA60C4E7996812
:101360000122A2401143F5E7740C002000E100E0E7
:10137000003C014020F00F03F0B500F00F041D68A1
:1013800067000326BE4025EA06051D601D6802228F
:10139000072C02FA07F242EA050294BF0024012456
:1013A0001A6003EB840300F007001A6A80000F2420
:1013B000844022EA04021A621A6A01FA00F0104319
:1013C0001862F0BD20F00F0200F00F0301209840DA
:1013D00080B21083704720F00F0200F00F0301204D
:1013E000984080B2508370472DE9F0410F4D104F67
:1013F0006E692A68002416404FF0010808FA04F3C9
:101400001E4206D06B6107EBC40357F834205868BE
:1014100090470134102CF1D1064B1B681BB1BDE87D
:10142000F041FFF7FDBBBDE8F08100BF003C01408B
:10143000740C00202C04002008B50B699A070ED507
:10144000CB6823F00203CB600B6923F002030B612E
:10145000224B002103EBC00253F8303034E00B691B
:101460005B070ED5CB6823F00403CB600B6923F038
:1014700004030B61194B012103EBC00253F8303018
:1014800022E00B691A070ED5CB6823F00803CB6066
:101490000B6923F008030B61104B022103EBC00220
:1014A00053F8303010E00B69DB060FD5CB6823F022
:1014B0001003CB600B6923F010030B61074B03EBA8
:1014C000C00253F83030032150689847044B1B6822
:1014D0001BB1BDE80840FFF7A3BB08BDF40C00201A
:1014E0002C04002018B101282FD1194B01E04FF036
:1014F0008043032929D8DFE801F0020B141D5A6349
:101500001A6922F002021A61DA6842F0020219E056
:101510009A631A6922F004021A61DA6842F004023E
:1015200010E0DA631A6922F008021A61DA6842F000
:10153000080207E01A641A6922F010021A61DA68D8
:1015400042F01002DA60002070474FF0FF30704721
:10155000000C004018B1012805D1044B01E04FF008
:101560008043586A70470020704700BF000C00405D
:1015700010B1012803D070474FF0804200E0034AC9
:10158000136843F001031360704700BF000C004074
:1015900010B1012805D07047044B4FF080521A60FB
:1015A0007047024B4FF480225A60704700E100E020
:1015B00038B5054698B1012839D11E4C206C40F051
:1015C000080020641C48102480F8324300F11450B5
:1015D00000F55C40B0FBF1F01849013811E0154C02
:1015E000206C40F0010020641348102480F81C4354
:1015F00000F1145000F55C40B0FBF1F04FF0804179
:10160000013888620E48002440F8352000EBC50000
:101610000C604C6043604B6943F001034B6128460A
:10162000FFF7B6FF2846FFF7A3FF204638BD4FF06F
:10163000FF3038BD0038024000E100E0000C0040FF
:10164000F40C00204FF080410020FFF7F5BE0000B1
:1016500001490120FFF7F0BE000C00402DE9F04FDA
:101660002D4B2E4A1B882E492E48DFF8CC90DFF8F0
:10167000CCA0DFF8CCB08BB00126ADF8243003F05D
:10168000F9F8FEF7A9FE0546FEF7BCFE0446FEF794
:10169000B5FE2A46009023464FF40071224803F01D
:1016A000E9F825EAE5754FF4007759F826401CB3B0
:1016B00094F80480E26A5AF82830606A0793174465
:1016C0000692FFF7DFFA069AB4F90610079B101A84
:1016D00022680592626A04920390E26A0292627939
:1016E000019209AAB8F1080FC8BF0132009205445F
:1016F000A26A584603F0BEF80136212ED5D10B4B15
:1017000002958DE888000A4A0A48194603F0B2F8A3
:101710000BB0BDE8F08F00BF685C00086A5C000891
:10172000705C0008755C0008BB5C0008415D000847
:10173000435D0008475D0008740400202402002077
:10174000055D0008042808D8DFE800F0030A0F143C
:1017500019000D4A136C19431164BFF34F8F704782
:10176000094B5A6C11435964F7E7074B1A6B114345
:101770001963F2E7044B5A6B11435963EDE7024BCF
:101780009A6B11439963E8E70038024070B514463C
:101790001CB18568C3689D4201D1101B70BD86686D
:1017A0000568731C83604368013B3340013CEB5C7C
:1017B00001F8013BECE7C268436830B58468121B4E
:1017C0009A4208D0C2680468013B1340551CC560AA
:1017D000E154002030BD4FF0FF3030BD37B5094C2B
:1017E00043F25645684601F0C3FBBDF80230AB42F8
:1017F00004D101980368DB689847F3E7204603F0BB
:10180000ADF8EFE7F95D000807B581B90C4B019021
:1018100043F25642B3F90010ADF80220684601F0D9
:1018200085FB002807DC074803F098F803E002294D
:1018300004D100F091FA03B05DF804FB0248F3E72D
:10184000040D0020B85D0008DF5D000810B51A48DF
:101850001A4CA4B003F082F8FFF786F8002118486C
:1018600003F008F81749204600F080FB164B636030
:10187000236820469B689847144B029300230193EA
:10188000134B0093062208234FF4C0611148FFF761
:1018900001FA114B0028188007DD104803F05EF8AC
:1018A000802204A90E4802F039F90E4803F056F8D8
:1018B000012024B010BD00BF285E0008080D0020E4
:1018C000455E0008145E0008091800086E5E0008F6
:1018D000DD1700083C0D0020040D00209D5E00086F
:1018E000D05E00087A5E00082DE9F04114462746D4
:1018F00001347B78002BFAD106464FF0010C3C787E
:10190000A4F130055FFA85F8B8F1090F07F1FF3E41
:1019100005D9A4F14105052D07D8A4F13705964551
:101920000AD2002419E07746E9E7A4F16105052D04
:1019300038D8A4F15705F2E7A7F1020E17F8017C99
:10194000A7F130045FFA84FCBCF1090F05D9A7F1B7
:101950004104052C07D8A7F1370401338B4209D97C
:101960000020BDE8F081A7F16104052CD9D8A7F1CA
:101970005704F2E745EA041434704FF0000C0136C6
:101980007245D0D9BCF1000FEAD1013E864202D89F
:101990001846BDE8F0813278017806F8011900F8A0
:1019A000012BF3E7BCF1000FDAD14FF0010CE7E7B0
:1019B0007FB53423694A43439C189B5801466848C5
:1019C0001D6902F057FF022104F10E0000F0B2FA87
:1019D000644802F04FFF082104F1100000F0AAFA59
:1019E000A189614802F046FF02230DF1060204219D
:1019F0002046A847002805DA5C4802F0AFFF012026
:101A000004B070BDBDF80610594802F033FF022340
:101A10000DF1060205212046A8470028ECDBBDF8A1
:101A20000610544802F026FF02230DF10602092198
:101A30002046A8470028DFDBBDF806104E4802F01C
:101A400019FF08230DEB030207212046A847061EB5
:101A500006DD4A4802F00EFF314602A800F06AFA9D
:101A6000617E474802F006FF02230DF106021B21AA
:101A70002046A8470028BFDBBDF80610414802F009
:101A8000F9FE02230DF1060208212046A84700288E
:101A9000B2DBBDF806103C4802F0ECFE02230DF16B
:101AA000060219212046A8470028B4BF3748384805
:101AB00002F054FF374802F0DDFE01230DF105026C
:101AC0000A212046A847002806DD9DF80530012B95
:101AD00002D1314802F0CEFE01230DF105020C21A6
:101AE0002046A847002806DD9DF80530012B02D1CD
:101AF0002A4802F0BFFE01230DF105021121204604
:101B0000A847002806DD9DF80530012B02D12448A6
:101B100002F0B0FE01230DF1050216212046A84770
:101B2000002806DD9DF80530012B02D11D4802F08A
:101B3000A1FE01230DF1050217212046A847002828
:101B400006DD9DF80530012B02D1174802F092FE08
:101B5000164802F003FF002052E700BF080D0020E6
:101B6000305F0008445F0008545F0008625F0008AF
:101B7000685F0008875F0008A35F0008B55F000882
:101B8000CC5F0008E45F0008F25F00080460000812
:101B90000F60000817600008216000082B60000833
:101BA000356000083B60000845600008DA5B00080B
:101BB00008B50020FFF7FCFE002008BD2DE9F04726
:101BC00096B006AF002304280D46BB803ED0052802
:101BD0000AD18A6892B1107818B10221381DFFF736
:101BE00083FE013801280BD92968474802F042FEDC
:101BF000012420464037BD46BDE8F0871046F0E797
:101C0000BB885BBABB800326686802F093FB55F87B
:101C10002620B30004469946002AE5D01378002B0D
:101C2000E2D0082107F11000FFF75EFEB0F10008D6
:101C3000DADD4D44BB8868683B81E94644B1214602
:101C4000324802F017FE0124CD46D2E70226DBE738
:101C50002F4D3862AE7E02F026FF3B89786206F097
:101C6000280646F00106AA8903B93A816B8BBA812E
:101C700003F00403002B274BA3F102012B7E03F199
:101C800001002876049303963B89ADF80830BB89A0
:101C9000ADF8043001F1020007F1280A1ABF01462D
:101CA00008220222CDF8008007F11003504601F00F
:101CB00087F9002803DA184802F050FEC3E7F861FC
:101CC0002B681448C7F818A01B68022207F11801F6
:101CD00010389847002801DA1048EDE7796A104873
:101CE00002F0C8FD414607F1100000F023F90D484D
:101CF00002F0C0FD07F10800022100F01BF90A48BC
:101D000002F02CFEA0E700BF4C60000875600008E0
:101D1000080D0020180D002095600008B56000082F
:101D2000CE600008E8600008665F00089368013B29
:101D3000002B10B4936008DA9469A34202DBCBB2A3
:101D40000A2B02D110BC02F061BF1368581C10604E
:101D50001970C8B210BC70472DE9F0475C4F5D4C5C
:101D60000546386888B082680A21FFF7DFFF2B68D4
:101D70007F225E68214601AB2846B0478046204658
:101D800001F0A0F9064628B9534802F0E7FD08B073
:101D9000BDE8F08703AA06A9204601F005FA02AAC9
:101DA000814604A9204601F0AFF9237803F0070328
:101DB0000546032B70D8DFE803F002696B6D4748D6
:101DC000DFF86CA102F0CAFDBDF80C10444802F027
:101DD00051FD494606A800F0ADF8BDF8081041488D
:101DE00002F048FD294604A800F0A4F83E4802F09D
:101DF00041FD237818074CBF3C483D4802F03AFDAE
:101E00003C4802F037FD2378D9064CBF37483848A4
:101E100002F030FD384802F02DFD23789A064CBFC1
:101E20003248334802F026FD344802F023FD23787F
:101E30005B064CBF3248334802F090FD324802F056
:101E400019FD61783148C1F3011102F013FDA17849
:101E50002F4802F00FFD44F210230022A8EB0601E8
:101E6000A01901F0DDFA2B4802F004FD3546C6F159
:101E70000109A84512D8284802F0FCFC9DF805206D
:101E80009DF80410254802F0F5FC80E7244897E708
:101E9000244895E7244893E7244891E7615D386832
:101EA000A1F120035F2B88BF3F218268FFF73EFF2F
:101EB00009EB05014A22B1FBF2F302FB1313012BDC
:101EC00004D1AE4202D0504602F0D4FC0135D0E736
:101ED000500200203C130020F0600008136100084D
:101EE0002E6100084F6100086F6100087B610008E7
:101EF0007F61000883610008916100089C6100080F
:101F0000A861000803630008AA610008B461000822
:101F1000B9610008C3610008D95B0008D0610008FE
:101F20001A610008316000081F610008266100087E
:101F3000C96100082DE9F0410A4FDFF82C80054601
:101F400046180446B44201D1BDE8F081AC4202D04B
:101F5000384602F08FFC14F8011B404602F08AFC60
:101F6000F0E700BF565A0008D262000838B50B4BA4
:101F70000446142240F81C3B0D4602F0BCFB08232B
:101F800084F8323000210F2384F8303084F8331085
:101F90006A78207FBDE8384001F0ACBCF0610008F1
:101FA00070B5044686B000F071F9204600F03BFEA3
:101FB00003AE0021217661830C22304602F0A6FB9D
:101FC000304601F0EDFE082505F0070306AA13448C
:101FD000715D13F80C2C01354A400C2D03F80C2CC4
:101FE000F2D19DF80C3023F00103314643F0020397
:101FF000082201A88DF80C3002F07DFB029A019BAB
:1020000012BA1BBA204600F095FCBDF8041049BA7C
:10201000204689B200F07FFC2046232100F0BBFC63
:1020200020461A2100F0AAFC2046002100F0D0FC36
:1020300020460122202100F044FD204601224FF4D9
:10204000807100F03EFD204600224FF4005100F068
:1020500038FD204601224FF4804100F032FD8022FD
:102060002946204600F07DF80421204600F092F831
:10207000042100F0FD02204600F073F80321204601
:1020800000F088F8032100F0F002204600F069F823
:10209000082220460E2100F064F80F21204600F0AF
:1020A00079F81621204600F086FD06B070BD10B507
:1020B000044600F0D4F80821204600F06BF808210F
:1020C00000F08002204600F04CF80121204600F08C
:1020D00061F80306F9D5C0F3801010BD10B590F873
:1020E00033300133044680F83330204600F0ABF83B
:1020F000A0F11103DBB2012BF7D9192818BF84F81E
:1021000032001921204600F056FD022384F83130B8
:1021100010BD70B51D4690F831306E1C1344144646
:1021200080F8313013460A46F1B200F04EF86019DB
:1021300070BD10B5012300F131020021044600F00A
:1021400044F802221146204600F00BF863683BB1C8
:10215000628B120504D520460321BDE810401847C4
:1021600010BD70B50446007F0D46164601F02EFCEA
:10217000206AFFF730F9324645F0C0010023207F86
:1021800001F08BFC206AFFF71DF9207FBDE870404D
:1021900001F02CBC37B50446007F0D4601F016FC5B
:1021A000206AFFF718F90DF10703002245F08001BE
:1021B000207F01F072FC206AFFF704F9207F01F014
:1021C00015FC9DF8070003B030BDF8B50446007F4C
:1021D0000F4615461E4601F0F9FB206AFFF7FBF893
:1021E0003A4600234021207F01F057FC3346294620
:1021F0000022207F01F030FC206AFFF7E3F8207F07
:10220000BDE8F84001F0F2BB10B50446007F01F0D4
:10221000DDFB206AFFF7DFF8207F00222021BDE8E8
:10222000104001F0F3BB1346007F0A46002101F085
:1022300013BC10B50446006AFFF7C4F8207FBDE860
:10224000104001F0D3BB08B590F830300F2B04D00C
:102250000121FFF79FFF00F01F03184608BD10B5CE
:102260000446FFF7F0FF0F280FD1A06AFFF7B3F87D
:1022700000214FF4967001F0A9FD01212046FFF7DF
:1022800089FF00F01F0084F8300010BD10B504462F
:10229000FFF7E5FFE06AFFF79EF80021012001F05B
:1022A00095FDE06AFFF78EF800211A20BDE8104086
:1022B00001F08CBD10B5032202210446FFF751FF47
:1022C0002046FFF7C0FF0828FAD110BD38B50446F4
:1022D000FFF7C5FF2046FFF7B6FFA0F11103DBB201
:1022E000012B0546F6D92046FFF7E4FF08212046DA
:1022F000FFF750FF637E00F0E00203F01F0320466B
:102300001A430821FFF72DFF29462046BDE8384033
:1023100000F051BC43680BB1002118477047000022
:102320002DE9F0470446884616461F46FFF78BFF07
:102330008146002C00F0D7800F2840F0D98020463D
:10234000FFF78DFFB8F11C0F1AD8DFE808F03F192E
:102350000F2E191937195819979E88198E19611956
:10236000A2A6AAAE19B2B6191951C400022F00F2E2
:1023700001813188204600F0CEFAB9F10F0F0CD15F
:10238000B8F1100F09D06FF085050F21204600F03D
:1023900012FC15F1860F40F0A8803B4632464146BC
:1023A0002046BDE8F04700F0D1BF082F00F2E280E0
:1023B000D6E90023204600F0BDFADEE7022F00F246
:1023C000D9803188204600F0E6FAD6E7022F06D001
:1023D0006FF01505B9F10F0F40F08780D5E7317820
:1023E000A1F10B030F2BF3D8204600F0C7FAC4E786
:1023F000022FEDD13378002BEAD10225EAE7022F34
:1024000000F2B880B6F90010204600F0E1FAF4E7D7
:10241000012F00F2B2803378013B042BADD801A22A
:1024200052F823F039240008452400087B230008D3
:1024300049240008572400080F21204600F0BBFB68
:10244000012552E01621F8E7638B5A05F8D520469E
:10245000FFF76FFEF4E72046FFF7A2FDF0E73278C2
:102460002021204600F02DFB87E7012F00F282801B
:102470003178204600F0C1FA0125ABE732784FF4FD
:102480008061204600F01DFBF6E732784FF40071C2
:10249000F7E732784FF40051F3E732784FF4804198
:1024A000EFE732784FF40061EBE732784FF4805178
:1024B000E7E732784FF48071E3E7012F5AD831789B
:1024C000052957D8638BDB057FF557AF49B2204606
:1024D00000F0AEFAD0E7012F4CD896F90010204654
:1024E00000F0E3FAC8E76FF012052846BDE8F08770
:1024F000B8F11C0F3FF651AF01A353F828F000BF0D
:10250000CD2300089B2300086D230008AB2300089F
:102510009B2300089B230008BD2300089B23000881
:10252000FF2300089B2300087D2400088B2400085B
:102530005F2400089B2300086B2400089B230008ED
:10254000112400089B230008932400089B24000802
:10255000A3240008AB2400089B230008B324000830
:10256000BB2400089B2300089B230008F1230008DC
:10257000D72400086FF08A052CE76FF08A05B4E7CE
:102580002DE9F0410446FFF75EFE0F2806464CD0C9
:102590000F212046FFF7FEFD022107462046FFF7E8
:1025A000F9FD7B07054603D563680121204698475E
:1025B00038073AD5162E01D0112E08D1638B590455
:1025C00033D5636802212046BDE8F0411847192E33
:1025D00001D0122E29D194F833301BB914490320AD
:1025E000FEF7B6FA013BDBB284F8333023B994F836
:1025F0003210204600F0DFFA6368B3B1628BD20478
:1026000013D505F0E005202D09D002D83DB1BDE875
:10261000F081602D07D0A02D03D0BDE8F08104210A
:10262000D1E70521CFE70621CDE7BDE8F08100BF66
:102630009B5B000813B504460121006AFEF7F4FD18
:10264000206AFEF7BFFE0121A06AFEF7EDFDA06A39
:10265000FEF7C1FE0121E06AFEF7E6FDE06AFEF743
:10266000B1FE0C4B009401220021606AFEF716FEB9
:102670002046FFF7F4FD1C212046FFF78BFD0328C1
:1026800005D12046FFF78CFC002002B010BD4FF0B2
:10269000FF30FAE7152300082DE9F34104460F4601
:1026A00090461E46FFF7B0FD01220DF107012046BE
:1026B000FFF7B9FD9DF8075005F07F05023D1FB9F2
:1026C0002046FFF7B6FD06E0454508D92046FFF74E
:1026D000B0FD6FF06805284602B0BDE8F0812A46DB
:1026E00039462046FFF79FFD022200212046FFF7D2
:1026F0009AFD002EE4D00122B1182046FFF793FD89
:102700002046FFF796FD07212046FFF743FD307076
:10271000E1E72DE9F04107460D469046FFF7DEFC64
:1027200000263446464508D17B8B5B0502D43846EB
:10273000FFF7FFFC2046BDE8F0816A68A31C134444
:102740007F2B05F1080508D8234655F8081C3846A4
:10275000FFF7DFFC01360446E4E76FF08A00BDE8CE
:10276000F081000008B5FFF76EFD0F38C0B20A28EF
:102770009ABF024B185C022008BD00BFE46100084C
:102780002DE9F8430F46164698460546002800F006
:102790009480A1F10903122B48D8DFE803F0172534
:1027A0002F474747471D4733373B3F474347474737
:1027B0000A00B8F1010F40F283800023737000F02B
:1027C000E8F8307002242046BDE8F883B8F1010F24
:1027D00076D966233380F5E7B8F1000F70D0FFF7A4
:1027E000C1FF30700124EEE7438B13F4806F02D0F9
:1027F00001243470E7E700233370F3E7438B13F4CD
:10280000007FF4E7438BC3F34033F5E7438BC3F317
:102810008033F1E7438BC3F3C023EDE7438BC3F36E
:102820000033E9E7438BC3F30023E5E74346324631
:1028300000F0F0FC10F1860F0446C4D12846FFF7E3
:1028400002FD0F2881463ED12846FFF708FD0E2FD6
:102850001AD008D8012F20D0082F3CD00F212846AD
:1028600000F0A9F9AFE7182F20D01C2FF6D1B8F14E
:10287000000F33D0284600F00EF90BE0284600F098
:102880009BF8022430802BE0B8F1000F26D02846B8
:1028900000F0ACF83070012422E02846FFF707FC76
:1028A000012408B134701BE0307019E0B8F1000F5A
:1028B00014D0284600F0B5F8ECE76FF0120482E778
:1028C0006FF08A047FE70E2FDED00ED8012FE4D000
:1028D000082F7FF478AFB8F1010FCFD86FF08A04DA
:1028E000B9F10F0F7FF46FAFB8E7182FDED01C2FB0
:1028F000BDD068E738B50A460C4602210546FFF709
:1029000030FC162C02D185F8304038BD2846FFF740
:102910009AFC8442F6E710B50A0A04468173C27332
:102920002021FFF71EFCA27B20462121BDE810409C
:10293000FFF717BC2DE9F843054616461F4600F180
:10294000100800246FF00709E2003046394601F014
:1029500067FA09FB04F208F8010B383230463946B1
:1029600001F05EFA04F12401C2B2C9B22846013472
:10297000FFF7F7FB082CE7D1BDE8F883A1F10B02C4
:102980000F2A05D8427E8A4202D04176FFF79EBCCC
:1029900070470020704737B50D0A8181CAB22221E5
:1029A0000446FFF7DEFB2A462321204603B0BDE89C
:1029B0003040FFF7D6BB000008B50521FFF7EAFB62
:1029C000024B00F00F0033F9100008BD1E62000832
:1029D000113109B21429A8BF142121EAE171024B77
:1029E0005A5C0521FFF7BDBB0862000808B52C2121
:1029F000FFF7D0FBC0F3071008BD38B50C462C21FB
:102A00000546FFF7C7FB072C28BF072400F00F007F
:102A100040EA0412D2B228462C21BDE83840FFF724
:102A2000A0BB08B52C21FFF7B5FBC0F3420008BDE1
:102A30000529A8BF0521002938B50C46A8BF0C46BA
:102A40004FF02C010546B8BF0724FFF7A3FB20F089
:102A50000E0040EA4402D2B228462C21BDE838409C
:102A6000FFF77FBB38B505460C4699B10A782D2192
:102A7000FFF777FB2E212846FFF78CFB637800F0E9
:102A8000F80203F007031A4328462E21BDE8384018
:102A9000FFF767BB38BD08B50921FFF77BFB00F0E6
:102AA0000F0040005B3840B208BD0029C4BF494256
:102AB00049B25B31C1F3430242F0C0020921FFF782
:102AC00050BB10B5438B0446002A40D00B43B1F5F0
:102AD000807F43830AD002D8202929D010BDB1F5C8
:102AE000007F12D0B1F5005F29D010BD00F11001B8
:102AF000FFF7B8FF04212046FFF79AFF53222F214A
:102B00002046BDE81040FFF72CBB2E21FFF742FB0B
:102B100040F01002D2B22E212046FFF722FB1721EF
:102B20002046FFF737FB40F00202D2B21721E7E759
:102B30002E21FFF72FFB00F0EF022E21E0E70E2100
:102B4000FFF728FB40F00402D2B20E21D8E723EAB7
:102B50000103B1F5807F43830AD002D820291CD01D
:102B600010BDB1F5007F09D0B1F5005F1CD010BDDC
:102B70004FF0FF31BDE81040FFF75ABF1721FFF7B4
:102B800009FB172100F0FD022046FFF7EAFA638BEC
:102B90009B060FD52E212046CBE72E21FFF7FAFA10
:102BA00040F01002D2B2C8E70E21FFF7F3FA00F0AE
:102BB000FB02CAE710BD38B504460D46FFF743FBDC
:102BC000A0F11103DBB2012B1AD91F2818D0A8429B
:102BD00028D0162816D1192D03D109212046FFF738
:102BE00089FE0F2D18D12046FFF764FB29462046A9
:102BF000FFF7D0FAA06AFEF7E5FB84F8305038BD45
:102C00002046DBE7192801D1162DE5E70F28E8D18A
:102C10002046FFF724FBE4E729462046BDE838407C
:102C2000FFF768BE38BD10B50446FFF718FB204615
:102C3000FFF709FB1F28FAD02046BDE81040FFF738
:102C400039BB000070B504460D46FDF719FC23683A
:102C500006463BB94FF0FF332360FDF719FC012511
:102C6000284670BDC5B10E4B1D6802212846FDF7F0
:102C7000FDFA236801330AD105F10803236000231C
:102C8000AB603046FDF704FCFDF7C4FBE7E72946DF
:102C90002046FDF7DFFFF4E7FDF7FAFBE0E700BFB2
:102CA0002804002070B50446FDF7EAFB25680646B7
:102CB0001DB9BDE87040FDF7EBBB6B1C02D10023D2
:102CC0002360F6E728460A2150F808392360FDF70B
:102CD000CDFA236813B94FF0FF33236015F8034C86
:102CE0003046FDF7D5FB2046BDE87040FDF7FEBA43
:102CF000F8B505460E46FDF7C3FB364B364A1B8832
:102D00001BB2074652F823301A6A002A4ED05C697B
:102D10009969A1424AD9611C5961D9690C4046B9E7
:102D2000196931B9611C04D13846FDF7B1FB204661
:102D3000F8BD002C3EDB02EBC40103C985E80300AB
:102D40001E69002E38D031681961002C1EDA7368B4
:102D500093E8030085E8030016F8043C052B23D014
:102D6000002373600A21A6F10800FDF77FFA16F828
:102D7000034C3846FDF78CFB0E2C28D82046FDF777
:102D8000B5FA24E03846FDF783FB20E09D695969D8
:102D9000D869691A8842A9BF691C4FF0FF35054000
:102DA000996102EBC505D2E70F24E2E74FF0FF344B
:102DB000002EB5D0DD60C3E7002CE3DA184603210E
:102DC000FDF754FA3846FDF763FBFDF723FB0124BA
:102DD000ADE700BF240400207404002010B583690F
:102DE0004469C2691C1BA24201DA002010BD5C1CB0
:102DF00013408461F9D4026A03C902EBC30383E878
:102E00000300012010BD00002DE9F8431E46264BAB
:102E100053F82150254B1B880380074691463DB946
:102E20003046FDF735FB4FF0FF342046BDE8F88310
:102E30002B79032B2ED01E4B01462846D3F8008059
:102E4000FFF7CCFF044650B13046FDF721FB98F860
:102E50000430052B01D1FDF7DDFA0124E5E7B9F1D6
:102E6000000F03D13046FDF713FBDEE798F804307E
:102E7000C8F80C70052B0CBF052104214046FDF756
:102E8000F5F9414605F11000FDF7E4FE3046FDF787
:102E9000FFFAE0E703C8EB6883E803000A2128464D
:102EA000FDF7E4F9F2E700BF7404002024040020D9
:102EB0002804002038B50446FDF7E2FA074B1B88CA
:102EC0002380074B214605461868FFF787FF044615
:102ED0002846FDF7DDFA204638BD00BF2404002057
:102EE0002804002008B50F4B53F82130B3B121223C
:102EF00002801A79032A0BD103C8DA6882E803003A
:102F000018460A21FDF7B2F9074B0120186008BDE9
:102F100001461846BDE80840FFF760BF4FF0FF309C
:102F200008BD00BF740400202C04002070B50446C6
:102F30000D46FDF7B0FA28B129462046BDE870409D
:102F4000FFF7D0BF094B1B881BB29D4204D120461E
:102F5000BDE87040FFF7AEBFFDF792FA2946034681
:102F600001222046BDE87040FFF74EBF2404002038
:102F70000121FFF7BDBE00000F4BD3F8882042F4BB
:102F8000700210B5C3F888204FF000629A600B4CB5
:102F9000102283F822200021DA77601801315229AB
:102FA00080F80023F9D11A6942F010021A615A69B7
:102FB00042F400725A6110BD00ED00E000E100E053
:102FC000F8B504460F461E4610219DF82430069899
:102FD00023706170154602B1B7B100B1A6B113F00C
:102FE000050F02D00DB9002869D09DF82830A370D4
:102FF000002861D09DF82030E37002289DF8213030
:10300000237103D0082827D00020F8BD02462C49A0
:10301000304601F061FB18B9237823F020032370B8
:10302000637843F008036370737863713378A37136
:103030000720002D43D0BDF81C20BDF820309A4257
:1030400017D1237843F040032370022D1AD0082DA6
:1030500023D0002DD8D1F8BD1C236370221D06F1AA
:10306000080313F8011D02F8011FB342F9D10D2026
:10307000DFE7431C9DF81C2022549DF81D20E254DC
:103080000230E2E7637863F07F0363707A7822545A
:10309000431C3A78E2540230F8BD637863F03F0392
:1030A000637007F10803044413F8012D04F8012BA1
:1030B000BB42F9D10830F8BD0320002DD9D1F8BDAD
:1030C0003E620008427802F00C03082B014611D042
:1030D0000C2B11D0B3B90078400613D4032012F0A2
:1030E000C00210D00B785B0658BF0230802A05D191
:1030F000023070470720F2E70D20F0E7C02A01D127
:10310000083070470020704770B501B11AB92549E1
:103110000320FDF71DFD437803F00C03082B08D1B5
:1031200003785C0603D5C3781370037953700723C3
:1031300012E00C2B08D103785B0603D5C37813701B
:10314000037953700D2307E013B16FF0150070BDC4
:1031500003785E06F9D40323447814F0C00411D038
:1031600005786D0605D4C65C16705D1C0233455D9E
:103170005570802C08D1C25C4A70184443780B709B
:10318000022070BD204670BDC02CDED1184401F174
:10319000080310F8012B03F8012D9942F9D10820FA
:1031A00070BD00BF9B5B000808B501B11AB9184992
:1031B0000320FDF7CDFC437803F00C03082B09D165
:1031C000C37813700379537043794B7083790B7014
:1031D000022008BD0C2B0ED1C378137010F8043FE9
:1031E000537001F1080310F8012F03F8012D8B42F1
:1031F000F9D1082008BD3BB9037813F0400F14BF84
:103200006FF01500002008BD6FF0150008BD00BF6D
:103210009B5B000810B5044610461A2900F2908006
:10322000DFE801F0338E0E1C25252F4F8E8E8E8EFB
:103230008E398E8E8E458E8E8E8E8E8E8E8E4B001D
:10324000012B03D840490320FDF782FC022204F140
:103250000E0101F050FA0223184610BD072BF1D9D8
:10326000082204F1100101F046FA0823F4E7022BCA
:10327000E8D1628B520702D508220280ECE7038076
:10328000EAE7022BDED1A289F7E7022BDAD1637ECF
:1032900003800123E0E7012BD4D1638B13F0200FCF
:1032A00002D001230370D7E700230370F1E7012B5D
:1032B000C8D1638B13F0020FF2E7022BC2D10322B5
:1032C000DBE7072BBED9638B5B074CBF08230223C8
:1032D0004FF000024CBF04F1100104F10E01042B69
:1032E0004270027018D0082B03D0022BBDD11346B8
:1032F00019E00A7882F0020202704A7842708A78F5
:103300008270CA78C2700A7902714A7942718A79E8
:103310008271CA79C2719FE70B7883F00203037050
:103320004B7843700223FF240022C470FE24827075
:1033300004714271CA5C827119444B78C37194E77D
:103340006FF0850388E700BF9B5B000870B51546EA
:103350001C4611295ED8DFE801F0095D15253535D9
:10336000455D5D5D5D5D5D4A5D5D5D54022C03D034
:103370002A490320FDF7ECFB1388FF2BF8D843768E
:10338000204670BD022CF3D800F10E060222002167
:10339000304601F0BBF922462946304601F0ABF930
:1033A0000224EDE7082CE3D800F1100608220021E2
:1033B000304601F0ABF922462946304601F09BF930
:1033C0000824DDE7022CD3D11388022B05D0082B6B
:1033D000D6D1438B43F0040302E0438B23F0040374
:1033E0004383CDE7022CC3D113888381C8E71278C9
:1033F000438B1AB143F020034383D1E723F020032A
:10340000FAE71278438B12B143F00203F4E723F09A
:103410000203F1E76FF08504B2E700BF9B5B000891
:103420002DE9F04F8DB000AF1E4613F400538146D6
:103430000D469046C7F810D0FB602BD106F0F7047C
:10344000102C27D005D8022C26D0042C06D004241A
:1034500004E0202C20D0802CF9D10824002D59D054
:1034600006F4404ABAF5804F18D0BAF5004F18D08C
:10347000BAF1000F05D1A649052207F11C0001F0A1
:103480001AFBFB6883B1A349072207F1240001F06E
:1034900012FB1FE00124E1E70224DFE705229E4939
:1034A000EBE705229D49E8E743F6F7633340B3F5C0
:1034B000207F00F0BC8051D8802B00F08D8036D862
:1034C000042B00F093802BD8002B00F08280022B7D
:1034D00000F085804346002B00F0AF80A045C0F08F
:1034E000AF80B8FBF4F3B5FBF4F804FB18557B612F
:1034F0000DB108F10108BAF5404F04D0002107F1E1
:103500001C0001F0B7F9A346002506F48056A84533
:1035100040F09880D7F810D03437BD46BDE8F08F22
:10352000102B53D0202BD5D107227D49ADE7B3F521
:10353000017F7FD009D8B3F5007F75D040F2022219
:103540009342C7D1042277494BE0B3F5047F68D09A
:10355000B3F5087FBED10722734996E7B3F5906FA4
:1035600059D017D840F20442934257D009D8B3F546
:10357000806F4DD040F202429342ABD106226B499C
:103580002FE0B3F5826F40D0B3F5846FA2D106224D
:1035900067497AE741F20402934233D009D8B3F580
:1035A000805F29D041F20202934293D10622614901
:1035B00017E0B3F5815F1CD0B3F5845F1FD041F2F3
:1035C0001002934286D105225B495EE706225B49E1
:1035D0005BE708225A4958E709225A4955E75A49F0
:1035E000062207F1240001F0EDF973E70C22574998
:1035F000F7E70622564948E70722564945E70822D9
:10360000554942E70C225549EBE7052254493CE76E
:103610000722544939E70822534936E70C22534917
:10362000DFE70622524930E7072252492DE70922F7
:1036300051492AE708225149D3E71023984650E719
:10364000012350E7022C58D0082C00F0AD80012C4B
:103650005AD1FB68002B47D019F905100D293AD82B
:10366000DFE801F0073939393939392B2D35313750
:103670002F33434801F0FEF879697A696B1CB3FB7C
:10368000F2F201FB123208F1FF310AB18D4211D181
:103690003C487960BB6001F0EDF87968BB688D4209
:1036A00008D0BAF5404F05D0594607F11C0001F08B
:1036B000E1F8BB68A3441D4629E73348DAE73348FD
:1036C000D8E73348D6E73348D4E73348D2E733481E
:1036D000D0E73348CEE7002904DAC9B2314801F017
:1036E000C9F8C9E71F29F9DD26B119F9051007F155
:1036F0002400F4E719F80510F9E716B139F91510A7
:10370000F5E739F81510F2E759F82510EFE700BF93
:10371000406200084F620008456200084A620008E3
:1037200056620008EE620008D7620008C262000814
:10373000AD620008996200087F62000830630008EB
:103740005D620008656200086E620008766200082B
:10375000846200088A62000891620008A062000882
:10376000A8620008B3620008BA620008C9620008D3
:10377000D1620008DE620008E5620008F662000817
:10378000FF620008D95B0008056300080B630008AE
:1037900011630008176300081D6300082363000815
:1037A000296300082F63000807F12401004896E709
:1037B000366300088368DB0710B5044606D5C06889
:1037C000064BC0B253F821309847E060044B1B68A9
:1037D0001BB1BDE81040FDF723BA10BDC413002093
:1037E0002C0400202DE9F04F8BB020B101286FD0C0
:1037F0004FF0FF3069E03D4A019205230721029214
:103800000392049307930591089306220692099365
:1038100000210DF104080DF1100C4FF0030E0227EA
:10382000012607AC5CF8212058F821305000D3F86D
:1038300000B00EFA00FA6FEA0A090BEA090BC3F8A6
:1038400000B0D3F800B007FA00F04BEA000BC3F861
:1038500000B0D3F808B009EA0B0BC3F808B0D3F8EE
:1038600008B04AEA0B0AC3F808A0D3F804A006FA85
:1038700002FB2AEA0B0AC3F804A0D3F80CA009EA59
:103880000A09C3F80C90D3F80C90072A40EA090003
:10389000D4BF4FF000094FF00109D86003EB890352
:1038A000A2EBC902186A92000F2505FA02F920EA74
:1038B0000900186254F82150186A05FA02F2013121
:1038C000024303291A62ADD100200BB0BDE8F08F8E
:1038D0000D23074A04930F210523019202920392BC
:1038E0000793059108930E2290E700BF0000024065
:1038F00000040240F8B506460F46042A04D8DFE863
:1039000002F00D06101418004FF0FF30F8BD2C4BDC
:103910001C5C0534E4B286B1012E3ED06FF001008C
:10392000F8BD274B1C5C0434F4E7254B1C5C0234C7
:10393000F0E7234B1C5C0134ECE74FF4805101208D
:10394000FDF700FF01210220FDF7FCFE012102200E
:10395000FDF7F8FE01210220FDF7F4FE194D304677
:10396000FFF740FFEB69002023F40063EB61286060
:1039700068602B6843F440732B602B6843EAC404EF
:103980002C602B6843F004032B602B681F432F60CF
:103990002B6843F040032B60F8BD4FF480410020BA
:1039A000FDF7D0FE02210846FDF7CCFE02210846B5
:1039B000FDF7C8FE02210846FDF7C4FE024DCEE722
:1039C000396300080030014000380040012808B584
:1039D00007D8054B012103EB8000FFF733F90020E6
:1039E00008BD4FF0FF3008BDBC130020012808B50A
:1039F00006D8054B03EB8000FFF754F9002008BD03
:103A00004FF0FF3008BD00BFBC13002070B101288B
:103A10000ED1094B98688007FCD5D9609968C90711
:103A2000FCD5DB6802B1137001207047034BF1E74E
:103A30004FF0FF30704700BF0038004000300140B9
:103A400000210148FFF7B6BE0030014001210148C6
:103A5000FFF7B0BE003800402DE9F34106460D46A1
:103A6000174698460024444503D1204602B0BDE8DD
:103A7000F0810DF107025DB1295D3046FFF7C6FF09
:103A8000002807DB17B19DF807303B550134EAE702
:103A90002946F2E74FF0FF30E8E770B516461A46C0
:103AA00005461C46FFF7B2FF002802DA4FF0FF3050
:103AB00070BD224631462846FFF7A8FF0028F5DBF7
:103AC000012070BD0C4B0146186882689368013B69
:103AD000002B10B4936005DA9469A34208DBCBB2E3
:103AE0000A2B05D01368581C1060197010BC704761
:103AF00010BC01F08BB800BF5002002008B53E207A
:103B0000FFF7E0FF2020FFF7DDFF034B1B689868FD
:103B1000BDE8084000F0C4BC500200202DE98048F8
:103B200087B000AF81460E469346FFF7E7FFDFF808
:103B300058A2B0460BF1FF340025A8EB0603A342C0
:103B40000BDA894B186841684B68013B002B4B60CE
:103B500006DA00F00BFF002806DAFFF7CFFFE8E7F0
:103B60000B685A1C0A6018780D2801D00A281BD14E
:103B700000240D2088F80040FFF7A4FF0A20FFF77B
:103B8000A1FF4645E9D0334622462546204619780E
:103B9000202930D9222901D0272938D15C7804BBCB
:103BA000724800F0DBFED8E7082801D07F2812D148
:103BB0004645C2D008F1FF33082008F8015CFB60DD
:103BC000FFF780FF2020FFF77DFF0820FFF77AFF37
:103BD000FB689846B1E708F10103FB6088F8000034
:103BE000F4E75C2C0CD001331C788C42D6D1597888
:103BF0002029D5D801351978D1B103F8010BC6E7D2
:103C00009C1C9B780132002BCAD02346ECE7197824
:103C10005C290BD1591C5B780132002BC0D04B1CA6
:103C200049782229BCD02029F1D8E3E71946F6E7E4
:103C3000002D92D0AB000E3323F00703C7F80CD051
:103C4000ADEB030D6C464DF82510304690F800E0C2
:103C500003460130BEF1000FF8D0BEF1220F02D0B2
:103C6000BEF1270F00D1013344F82130184601334B
:103C700090F800E0BEF1000FF8D101318D42E5D19E
:103C8000201F1AB150F8043F002B3DD12268C7F81D
:103C90001090C7F814A0002307F1100151F82380F9
:103CA000B8F1000F3ED10133022BF5D12168304825
:103CB00000F0EFFE0546002851D12E4A2E492F482C
:103CC000DFF8B88000F0D6FD2D4800F047FE2C4606
:103CD000C7F81090C7F814A007F1100353F8245048
:103CE00025B10C350C3555F8181C91BB0134022C4C
:103CF000F2D12BE0BEF15C0F06D191F800E0BEF1ED
:103D0000000F08D1013AC1D0194613F801EBBEF1FA
:103D1000000FEFD1B5E791F801E001F801EBECE716
:103D200008F10C08D8F800000028BCD011467B60D0
:103D3000BA6000F0AEFEBA687B680028F0D1D8F80F
:103D40000830002BB2D0214628469847D7F80CD02F
:103D500003E755F8142C404600F08CFDC2E72168BB
:103D6000084800F087FDF1E7500200203B6300089F
:103D70005463000859630008656300086D63000818
:103D8000776300089F630008C063000808B5FCF76C
:103D900065FB002008BD08B5FDF760FC002008BDEC
:103DA0000C22014900F0A7BC107AFF1FFEF77ABF72
:103DB00038B504460020FDF7CDFB05460020FDF791
:103DC000C9FB401BA042F9D338BD000030B587B015
:103DD00004460D46FCF75FFB48B11DB10E490320B8
:103DE000FCF7B6FE2046FFF7E3FF07B030BD0B4BF4
:103DF000009003900290012168460493CDF814D0FE
:103E0000FEF720FF214601A82A46FCF751FE0121BA
:103E10006846FEF717FFE8E79B5B0008AD3D00082A
:103E2000D0400B1CD1409C46203AD340184352420C
:103E3000634693401843704780F0004002E000BFA3
:103E400081F0004142001FBF5FEA410392EA030F85
:103E50007FEA226C7FEA236C6AD04FEA1262D2EBCF
:103E60001363C1BFD218414048404140B8BF5B42D4
:103E7000192B88BF704710F0004F40F4000020F06D
:103E80007F4018BF404211F0004F41F4000121F083
:103E90007F4118BF494292EA030F3FD0A2F10102CD
:103EA00041FA03FC10EB0C00C3F1200301FA03F10B
:103EB00000F0004302D5494260EB4000B0F5000F2E
:103EC00013D3B0F1807F06D340084FEA310102F1ED
:103ED0000102FE2A51D2B1F1004F40EBC25008BF9F
:103EE00020F0010040EA03007047490040EB000069
:103EF00010F4000FA2F10102EDD1B0FA80FCACF198
:103F0000080CB2EB0C0200FA0CF0AABF00EBC25096
:103F100052421843BCBFD0401843704792F0000F84
:103F200081F4000106BF80F400000132013BB5E7D7
:103F30004FEA41037FEA226C18BF7FEA236C21D04D
:103F400092EA030F04D092F0000F08BF08467047B2
:103F500090EA010F1CBF0020704712F07F4F04D180
:103F6000400028BF40F00040704712F100723CBF93
:103F700000F50000704700F0004343F0FE4040F4BD
:103F8000000070477FEA226216BF08467FEA23637B
:103F90000146420206BF5FEA412390EA010F40F466
:103FA000800070474FF0000304E000BF10F00043B2
:103FB00048BF40425FEA000C08BF704743F0964399
:103FC00001464FF000001CE050EA010208BF7047B4
:103FD0004FF000030AE000BF50EA010208BF70473B
:103FE00011F0004302D5404261EB41015FEA010C50
:103FF00002BF84460146002043F0B64308BFA3F148
:104000008053A3F50003BCFA8CF2083AA3EBC25329
:1040100010DB01FA02FC634400FA02FCC2F1200248
:10402000BCF1004F20FA02F243EB020008BF20F07F
:104030000100704702F1200201FA02FCC2F12002E5
:1040400050EA4C0021FA02F243EB020008BF20EADA
:10405000DC7070474FF0FF0C1CEAD0521EBF1CEA08
:10406000D15392EA0C0F93EA0C0F6FD01A4480EAF6
:10407000010C400218BF5FEA41211ED04FF00063DF
:1040800043EA501043EA5111A0FB01310CF000400B
:10409000B1F5000F3EBF490041EAD3715B0040EA31
:1040A000010062F17F02FD2A1DD8B3F1004F40EB01
:1040B000C25008BF20F00100704790F0000F0CF0D4
:1040C000004C08BF49024CEA502040EA51207F3A98
:1040D000C2BFD2F1FF0340EAC250704740F4000073
:1040E0004FF00003013A5DDC12F1190FDCBF00F064
:1040F00000407047C2F10002410021FA02F1C2F112
:10410000200200FA02FC5FEA310040F1000053EAAD
:104110004C0308BF20EADC70704792F0000F00F0FB
:10412000004C02BF400010F4000F013AF9D040EA01
:104130000C0093F0000F01F0004C02BF490011F495
:10414000000F013BF9D041EA0C018FE70CEAD15393
:1041500092EA0C0F18BF93EA0C0F0AD030F0004C13
:1041600018BF31F0004CD8D180EA010000F00040C7
:10417000704790F0000F17BF90F0004F084691F085
:10418000000F91F0004F14D092EA0C0F01D14202BF
:104190000FD193EA0C0F03D14B0218BF084608D188
:1041A00080EA010000F0004040F0FE4040F40000D2
:1041B000704740F0FE4040F4400070474FF0FF0C65
:1041C0001CEAD0521EBF1CEAD15392EA0C0F93EAAC
:1041D0000C0F69D0A2EB030280EA010C49024FEAFE
:1041E000402037D04FF0805343EA111143EA1013B7
:1041F0000CF000408B4238BF5B0042F17D024FF46F
:10420000000C8B4224BF5B1A40EA0C00B3EB510F49
:1042100024BFA3EB510340EA5C00B3EB910F24BF32
:10422000A3EB910340EA9C00B3EBD10F24BFA3EBB7
:10423000D10340EADC001B0118BF5FEA1C1CE0D17F
:10424000FD2A3FF650AF8B4240EBC25008BF20F032
:10425000010070470CF0004C4CEA50207F32C2BF86
:10426000D2F1FF0340EAC250704740F400004FF023
:104270000003013A37E792F0000F00F0004C02BF54
:10428000400010F4000F013AF9D040EA0C0093F01E
:10429000000F01F0004C02BF490011F4000F013B78
:1042A000F9D041EA0C0195E70CEAD15392EA0C0FE0
:1042B00008D142027FF47DAF93EA0C0F7FF470AF18
:1042C000084676E793EA0C0F04D14B023FF44CAF5B
:1042D00008466EE730F0004C18BF31F0004CCAD1F0
:1042E00030F000427FF45CAF31F000437FF43CAF2C
:1042F0005FE700BF42000ED2B2F1FE4F0BD34FF08A
:104300009E03B3EB126209D44FEA002343F000434B
:1043100023FA02F070474FF00000704712F1610F6E
:1043200001D1420202D14FF0FF3070474FF0000040
:10433000704700BF0A22002100F052BC8A892DE993
:10434000F041054610070C465AD44B68002B05DC9B
:104350000B6C002B02DC0020BDE8F081E66A002E29
:10436000F9D0002312F480522F682B6033D0606D97
:10437000A3895A0705D56368C01A636B0BB1236C18
:10438000C01A00230246E66A216A2846B047431C49
:10439000A38906D129681D294BD82B4ACA40D607C4
:1043A00047D500226260D9042269226004D5421CEC
:1043B00001D12B6803B96065616B2F600029CAD0F9
:1043C00004F14403994202D0284600F0A7F90020E6
:1043D0006063BDE8F081216A01232846B047411C93
:1043E000C6D12B68002BC3D01D2B01D0162B01D1B9
:1043F0002F60B0E7A38943F04003A381BDE8F081BB
:104400000F69002FA7D093070E6808BF4B690F6094
:1044100018BF0023A6EB07088B60B8F1000F9ADDE8
:1044200043463A46216AA66A2846B047002807DC78
:10443000A38943F04003A3814FF0FF30BDE8F08132
:104440000744A8EB0008E8E70100402038B50B69F5
:1044500005460C46DBB118B183690BB900F072F860
:104460000C4B9C4209D16C68B4F90C307BB12146ED
:104470002846BDE83840FFF761BF074B9C4201D199
:10448000AC68F1E7054B9C4208BFEC68ECE7002004
:1044900038BD00BF4864000868640008286400084C
:1044A000014620B9044B0549186800F0D3B8044B05
:1044B0001868FFF7CBBF00BF886400084D440008B0
:1044C00050020020014900F0C5B800BF4D4400086B
:1044D000002310B504460360436083608181436616
:1044E000C281036143618361194608225C3000F098
:1044F0000DF9054B6362054BA362054BE362054B67
:104500002462236310BD00BF0D4A00082F4A000833
:10451000674A00088B4A000870B54A1E6825554353
:104520000E4605F1740100F047F9044640B1002140
:1045300080E842000C30A06005F1680200F0E6F867
:10454000204670BD836910B5044633BB8364C364E1
:104550000365124B124A1B688262984204BF012312
:10456000836100F01FF86060204600F01BF8A06037
:10457000204600F017F80022E06004216068FFF791
:10458000A7FF01220921A068FFF7A2FF0222122142
:10459000E068FFF79DFF0123A36110BD8864000858
:1045A000C5440008F8B51C4B1E68B369074613B92B
:1045B0003046FFF7C7FF4836B4687368013B03D540
:1045C000336833B13668F7E7B4F90C506DB168342D
:1045D000F4E704213846FFF79FFF30600028F1D14F
:1045E0000C233B6004462046F8BD4FF6FF73E38181
:1045F0000123A38165662560A5606560256165610D
:10460000A5610822294604F15C0000F07FF865638B
:10461000A563A564E564E6E7886400082DE9F04138
:10462000884600F14804002614B93046BDE8F08100
:10463000A5686768013F01D52468F5E7AB89012BC0
:1046400006D9B5F90E30013302D02846C0470643DB
:104650006835EFE72DE9F8438046894600F14804C4
:10466000002614B93046BDE8F883A5686768013FA5
:1046700001D52468F5E7AB89012B07D9B5F90E30D0
:10468000013303D029464046C84706436835EEE764
:1046900070B50D4E0D4CA41BA4100025A54209D1E8
:1046A0000B4E0C4CFBF770FDA41BA4100025A5427B
:1046B00005D170BD56F8253098470135EEE756F81C
:1046C000253098470135F2E7C8650008C86500083D
:1046D000C8650008C865000810B501390244904259
:1046E00001D1002010BD10F8013B11F8014FA34289
:1046F000F5D0181B10BD10B5431E0A44914200D1DD
:1047000010BD11F8014B03F8014FF7E702440346CF
:10471000934200D1704703F8011BF9E738B505460D
:10472000002945D051F8043C0C1F002BB8BFE418F9
:1047300000F0A2FB1F4A1368104633B9636014608F
:104740002846BDE8384000F098BBA3420CD9216848
:104750006218934204BF1A685B68636004BF521812
:1047600022600460ECE713465A680AB1A242FAD903
:1047700019685818A0420BD1206801445818824289
:104780001960DDD1106852685A6001441960D7E79A
:1047900002D90C232B60D3E7206821188A4204BF7A
:1047A00011685268626004BF091821605C60C7E745
:1047B00038BD00BFCC13002070B5CD1C25F003051B
:1047C00008350C2D38BF0C25002D064601DBA9420B
:1047D00003D90C233360002070BD00F04DFB234A49
:1047E0001468214691B9224C23681BB93046FBF767
:1047F000CFFC206029463046FBF7CAFC431C26D17B
:104800000C233360304600F038FBE4E70B685B1B99
:104810001AD40B2B0FD90B60CD50CC18304600F0BA
:104820002CFB04F10B00231D20F00700C31A1BD042
:104830005A42E25070BD8C420DBF63684B686360A2
:10484000136018BF0C46E9E70C464968CAE7C41C68
:1048500024F00304A04205D0211A3046FBF798FC4F
:104860000130CDD02560D9E770BD00BFCC1300204A
:10487000D01300200FB40A4B13B51C6824B1A369F0
:1048800013B92046FFF75EFE05AB049AA1680193B9
:10489000204600F06BFC02B0BDE8104004B0704749
:1048A0005002002070B50E46054618B183690BB959
:1048B000FFF748FEAB69AC6813B92846FFF742FE24
:1048C000234B9C4217D16C68A3891B071DD5236914
:1048D000DBB1013EA36816F8011F013BA360E9B9F3
:1048E000002B2EDA22460A21284600F08FF90130EB
:1048F00011D00A2070BD174B9C4201D1AC68E3E790
:10490000154B9C4208BFEC68DEE72146284600F0C4
:10491000CFF90028DDD04FF0FF3070BD002B04DA56
:10492000A269934206DB0A2904D023685A1C22603C
:104930001970CFE72246284600F068F90130C9D146
:10494000E9E723680A205A1C2260187070BD00BF76
:10495000486400086864000828640008024B0146A7
:104960001868FFF79FBF00BF5002002038B50C4603
:10497000054618B183690BB9FFF7E4FD0E4B9C4265
:104980000DD16C682146284600F0A6FE88B9636800
:10499000013B636023685A1C2260187838BD074BBE
:1049A0009C4201D1AC68EDE7054B9C4208BFEC6826
:1049B000E8E74FF0FF3038BD48640008686400083D
:1049C000286400080EB400B59CB04FF402711DAB12
:1049D000ADF81410029006906FF000410A4804915F
:1049E00007914FF6FF7153F8042BADF816100068CD
:1049F000019302A900F09EFA029B00221A701CB0DB
:104A00005DF804EB03B070475002002010B50C466F
:104A1000B1F90E10FBF7DAFB0028ABBF636DA38979
:104A20001B1823F48053ACBF6365A38110BD2DE92F
:104A3000F0411F468B89DB0505460C46164605D519
:104A400002230022B1F90E10FBF7CDFBA389B4F9C4
:104A50000E1023F48053A38132463B462846BDE81E
:104A6000F041FBF7B7BB10B50C46B1F90E10FBF7E0
:104A7000BAFB431CA38915BF606523F4805343F43C
:104A80008053A38118BFA38110BDB1F90E10FBF7AD
:104A9000A5BB10F8012B11F8013B012A28BF9A424F
:104AA000F7D0D01A7047034613F8012B002AFBD128
:104AB000181A0138704770B5044602B970BD234614
:104AC00011F8015B03F8015B561E1DB91444A342A3
:104AD00003D170BD1C463246EFE703F8015BF6E7F1
:104AE0002DE9F84F8046894692461F468B465D4623
:104AF0000A9815F8014B00F049F92044467816F061
:104B000008060BD12D2C0BD12C7801260BF10205B8
:104B100067B1102F14D1302C0AD011E0AB46E6E774
:104B20002B2C04BF2C780BF10205F1E7302C27D198
:104B30002B7803F0DF03582B4BD16C78102702350C
:104B4000002E0CBF6FF000414FF000410022B1FB7E
:104B5000F7FE104607FB1E1CA4F13003092B11D8E9
:104B60001C46A7421DDD531C07D0864516D301D134
:104B7000A44513DB00FB0740012215F8014BEBE7CE
:104B80000A27DDE7A4F14103192B01D8373CE8E7F8
:104B9000A4F16103192B04D8573CE2E74FF0FF3230
:104BA000EBE7531C08D12223C8F800300846BAF1BD
:104BB000000F07D1BDE8F88F06B14042BAF1000FEF
:104BC0000CD022B1013DCAF80050BDE8F88F4D4627
:104BD000F9E73024002FB3D10827B1E7BDE8F88FFB
:104BE000084B37B51C68084D236A002B08BF2B46BD
:104BF000009313460A4601462046FFF771FF03B0B3
:104C000030BD00BF50020020B4020020F8B50E46AF
:104C10001446054618B183690BB9FFF793FC214B85
:104C20009C422AD16C68A369A360A3891A072ED578
:104C3000236963B323692068C01A6369F6B2984296
:104C4000374604DB21462846FFF700FC28BBA36853
:104C5000013BA36023685A1C22601E706369013007
:104C6000984204D0A389DB0719D50A2E17D1214613
:104C70002846FFF7EBFB90B10FE00B4B9C4201D1B4
:104C8000AC68D0E7094B9C4208BFEC68CBE72146F3
:104C9000284600F00DF80028CCD04FF0FF373846FA
:104CA000F8BD00BF48640008686400082864000874
:104CB000324B70B51D6806460C4625B1AB6913B979
:104CC0002846FFF73FFC2E4B9C420FD16C68B4F98D
:104CD0000C309AB215072CD4D00611D409223260B8
:104CE00043F04003A3814FF0FF3070BD254B9C4241
:104CF00001D1AC68EBE7244B9C4208BFEC68E6E7C7
:104D0000510712D5616B41B104F14403994202D0BD
:104D10003046FFF703FD00236363A38923F02403D8
:104D2000A3810023636023692360A38943F0080300
:104D3000A38123694BB9A38903F42073B3F5007FE2
:104D400003D02146304600F049F8A28912F0010351
:104D50000CD00023A36063695B42A361236953B94C
:104D6000B4F90C3013F08000BAD170BD920758BF6F
:104D70006369A360F2E70020F7E700BF500200205C
:104D8000486400086864000828640008D0F8EC0053
:104D9000704770B50E46B1F90E10002990B0144658
:104DA0001D4607DA00232B60B3891A0610D44FF48E
:104DB00080630EE001AAFBF71BFA0028F2DB029ADF
:104DC00002F47042A2F500535A425A412A60EEE7BB
:104DD00040230020236010B070BD00008B8973B5A4
:104DE0009D0706460C4607D504F14703236023615F
:104DF0000123636102B070BD01AB6A46FFF7C9FFD2
:104E0000009905463046FFF7D7FC38B9B4F90C30A5
:104E10009A05EFD443F00203A381E5E70C4BB3629C
:104E2000A389206043F08003A381009B6361019B01
:104E300020614BB1B4F90E103046FBF7DEF918B122
:104E4000A38943F00103A381A3891D43A581D1E771
:104E5000C544000882B001B901A942B14BB1137831
:104E60000B601278101C18BF012002B0704710466A
:104E7000FBE76FF00100F8E7704770472DE9F04756
:104E80008E689E4282460C469146984635D88A895D
:104E900012F4906F31D0256809696F1A6569022391
:104EA00005EB450595FBF3F508F101033B449D42F5
:104EB00038BF1D46530531D52946FFF77DFC064610
:104EC00050B90C23CAF80030A38943F04003A381F2
:104ED0004FF0FF30BDE8F0873A462169FFF70BFC41
:104EE000A38923F4906343F08003A3812661656165
:104EF0003E44ED1B2660A5604646464528BF464613
:104F000032464946206800F0D3FCA3689B1BA3608F
:104F100023681E4426600020BDE8F0872A4600F082
:104F2000E1FC06460028E1D121695046FFF7F6FB77
:104F3000C7E700002DE9F04F9DB0804603938B89B1
:104F40001C060D4616460FD50B696BB94021FFF7BD
:104F500033FC2860286128B90C23C8F800304FF0D2
:104F6000FF30C5E040236B610023099320238DF8B7
:104F7000293030238DF82A304FF0010B37463C465C
:104F800014F8013B002B3CD1B7EB060A0BD053467B
:104F9000324629464046FFF771FF013000F0A380FA
:104FA000099B534409933B78002B00F09C8000231D
:104FB0004FF0FF3204930793059206938DF8533018
:104FC0001A9305222178504800F022FC671C049BAC
:104FD000D8B9D90644BF20228DF853201A0744BF00
:104FE0002B228DF8532022782A2A16D0079A0021E6
:104FF0000A20274601343B78303B092B51D9C9B1EF
:1050000011E0252BC0D02746B9E73F4A801A0BFA9A
:1050100000F0184304903C46D3E7039A111D126830
:105020000391002A01DB079204E0524243F002039D
:10503000079204933B782E2B0ED17B782A2B07F115
:10504000010132D1039B1A1D1B680392002BB8BFCC
:105050004FF0FF33023705932C4C3978032220465A
:1050600000F0D6FB38B14023001B03FA00F0049B8C
:10507000034304930137397825488DF82810062218
:105080007E1C00F0C5FB002835D0224BFBB9039BEA
:10509000073323F0070308330393099B4B44099319
:1050A0006CE700FB02320121A3E7002305931846B9
:1050B0000A240F4601313A78303A092A03D9002BE5
:1050C000CAD00590C8E704FB00200123F1E703AB39
:1050D00000932A46104B04A94046AFF30080B0F17C
:1050E000FF3F8146D9D1AB895B063FF538AF0998C0
:1050F0001DB0BDE8F08F03AB00932A46064B04A910
:10510000404600F0BFF9EAE7946400089A6400089A
:105110009E640008000000007D4E00089368013B7B
:10512000002B10B4936008DA9469A34202DBCBB27F
:105130000A2B02D110BCFFF769BD1368581C106020
:105140001970C8B210BC7047F8B506460F46144631
:10515000D518AC4201D1002007E03A4614F8011BF3
:105160003046FFF7DBFF431CF3D1F8BD2DE9F04FCC
:105170009DB00C4617460393064618B183690BB9D8
:10518000FFF7E0F97C4B9C4257D17468A38918075C
:105190005DD52369002B5AD00023099320238DF875
:1051A000293030238DF82A304FF0010BB8464546A0
:1051B00015F8013B002B55D1B8EB070A0BD053462D
:1051C0003A4621463046FFF7BFFF013000F0C48069
:1051D000099B5344099398F80030002B00F0BC80E1
:1051E00000234FF0FF3204930793059206938DF846
:1051F00053301A9305222978604800F009FB05F125
:105200000108049B002831D1D90644BF20228DF823
:1052100053201A0744BF2B228DF853202A782A2ABC
:105220002CD0079A00210A20A846013598F80030B2
:10523000303B092B6DD971B326E0514B9C4201D113
:10524000B468A3E74F4B9C4208BFF4689EE7214631
:105250003046FFF72DFD00289ED04FF0FF301DB0E7
:10526000BDE8F08F252BA7D0A846A0E7434A801AB7
:105270000BFA00F0184304904546BBE7039A111D52
:1052800012680391002A01DB079204E0524243F0C6
:1052900002030792049398F800302E2B10D198F84F
:1052A00001302A2B08F1010137D1039B1A1D1B681D
:1052B0000392002BB8BF4FF0FF3308F102080593AB
:1052C000314D98F800100322284600F0A1FA40B1B1
:1052D0004023401B03FA00F0049B0343049308F1AE
:1052E000010898F8001029488DF82810062208F1C6
:1052F000010700F08DFA002834D0254B03BB039B37
:10530000073323F0070308330393099B4B440993A6
:105310004CE700FB0232012186E700230593184683
:105320000A258846013198F80020303A092A03D925
:10533000002BC5D00590C3E705FB00200123F0E753
:1053400003AB00932246134B04A93046AFF3008011
:10535000B0F1FF3F8146D8D1A3895B063FF57DAF11
:1053600009987CE703AB009322460A4B04A9304618
:1053700000F088F8ECE700BF486400089464000877
:1053800068640008286400089A6400089E640008A5
:1053900000000000495100082DE9F04791461F46E2
:1053A0008A680B69DDF820809342B8BF1346C9F8BC
:1053B000003091F8432006460C4612B10133C9F87B
:1053C00000302368990642BFD9F800300233C9F88B
:1053D0000030256815F0060507D104F1190AE368C5
:1053E000D9F800209B1A9D4229DB94F843302268AB
:1053F000003318BF012392062ED404F1430239462C
:105400003046C047013021D02368E568D9F8002034
:1054100003F00603042B08BFAD1AA36822690CBF72
:1054200025EAE57500259342C4BF9B1AED184FF09D
:1054300000091A344D451BD10020BDE8F087012337
:10544000524639463046C047013003D14FF0FF3055
:10545000BDE8F0870135C2E7E1185A1C302081F819
:105460004300224494F8451082F843100233C4E705
:105470000123224639463046C0470130E6D009F1C3
:105480000109D7E72DE9F04317460A7E85B06E2A59
:10549000984606460C460C9B01F1430E00F0BC807A
:1054A0001AD8632A2ED00AD8002A00F0C880582AB9
:1054B00000F08A8004F1420584F842202AE0642A40
:1054C00001D0692AF6D121681A6811F0800F23D023
:1054D000111D1960136827E0732A00F0B48008D802
:1054E0006F2A2AD0702AE5D10A6842F020020A60A9
:1054F00003E0752A21D0782ADCD1782284F845206F
:105500006E4964E01A6801F14205111D19601368C3
:1055100084F842300123A3E011F0400F02F10401AE
:105520001960D7D0B2F90030002B03DA2D225B428C
:1055300084F8432062490A2217E02068196810F0B5
:10554000800F03D0081D18600B6806E010F0400FB4
:1055500001F104001860F7D00B8859496F2A14BF75
:105560000A220822002084F843006568A560002D07
:10557000C0F29C80206820F004002060002B3FD106
:10558000002D40F095807546082A0BD12368DA0774
:1055900008D5236962689A42DEBF302305F8013CD2
:1055A00005F1FF35AEEB05032361CDF800803B46E6
:1055B00003AA21463046FFF7EFFE013055D14FF0E8
:1055C000FF3005B0BDE8F08381F845203C492268F2
:1055D000186812F0800F00F104051D6001D0036807
:1055E00002E05506FBD50388D00744BF42F02002F5
:1055F00022601BB9226822F0200222601022B1E74B
:105600007546B3FBF2F002FB1033CB5C05F8013DAD
:1056100003460028F5D1B7E708681A68496910F011
:10562000800F04D0101D18601368196007E010F097
:10563000400F02F1040018601368F6D019800023AF
:1056400023617546B1E71A68111D19601568626813
:105650000021284600F0DCF808B1401B6060636858
:105660002361002384F843309FE723692A463946A3
:105670003046C0470130A2D023689B0707D50025DC
:1056800004F11909E368039A9B1A9D4205DBE0685F
:10569000039B9842B8BF184693E701234A46394610
:1056A0003046C04701308AD00135EBE7002BA7D147
:1056B0000B7884F8423004F1420565E7B6640008CF
:1056C000A5640008838903F00903092B01D1FEF7C3
:1056D000E7BE002070470000F8B50C46054618B13B
:1056E00083690BB9FEF72EFF3B4B9C420AD16C68D5
:1056F000B4F90C200023636093B29E060CD54FF0E2
:10570000FF30F8BD354B9C4201D1AC68F0E7344B1B
:105710009C4208BFEC68EBE7580748D4D90605D48B
:10572000092342F040022B60A281E8E71A070BD55B
:1057300021462846FEF78AFE0028E0D1A389A06012
:1057400023F00803A381A061A38943F00403A3818C
:1057500023691BB921462846FFF740FBB4F90C70BA
:10576000BEB2B3070FD00123A3811E4B1E49186898
:1057700006F00906FEF752FF092EA78103D1214644
:105780002846FEF7DBFD22692260666A6369216AAA
:105790002846B047002860601CDCA38917BF0022A0
:1057A00043F0200343F040036260A381A7E7616BED
:1057B0000029CDD004F14403994202D02846FEF7D7
:1057C000ADFF236C636000206063002BC0D0E36BEF
:1057D0002360F8BD0020F8BD486400086864000834
:1057E0002864000888640008C556000849B1FF2AEB
:1057F00085BF8A2303600A704FF0FF3098BF0120F5
:1058000070470846704700000000000000000000DC
:1058100001F0FF01102A2BDB10F0070F08D010F861
:10582000013B013A8B422DD010F0070F42B3F6D165
:10583000F0B441EA012141EA014122F007047FF07E
:1058400000070023F0E80256083C85EA010586EAD5
:10585000010685FA47F5A3FA87F586FA47F6A5FA11
:1058600087F68EB9EED1F0BC01F0FF0102F007021D
:1058700032B110F8013B013A83EA010313B1F8D1C8
:105880000020704701387047002D06BF35460338A9
:10589000073815F0010F07D1013015F4807F02BFE2
:1058A000013015F4C03F0130F0BC0138704700BF33
:1058B000884210B501EB020303D8421E99420CD175
:1058C00010BD9842F9D28118D21AD34200D110BD2E
:1058D00013F8014D01F8014DF7E711F8014B02F8FB
:1058E000014FEBE7F8B5074614460E4621B91146BD
:1058F000BDE8F840FEF760BF22B9FEF70FFF25466E
:105900002846F8BD00F014F884420FD921463846E5
:10591000FEF752FF05460028F2D031462246FEF738
:10592000EAFE31463846FEF7F9FEE9E73546E7E795
:1059300051F8040C0028A0F10400BCBF0B58C0189B
:105940007047425553204641554C542048414E44DF
:105950004C4552004445425547204D4F4E2048414A
:105960004E444C45520044554D4D592048414E44FB
:105970004C4552000A49535220737461636B206F87
:10598000766572666C6F77656400537461636B2033
:10599000706F696E74657220636F72727570746572
:1059A000642C20726573657420746F20746F70208E
:1059B0006F6620737461636B000A436F6E74657861
:1059C00074206265666F72652068617264666175D5
:1059D0006C743A0020202072303A2030782530381C
:1059E0006C780A20202072313A2030782530386CCB
:1059F000780A20202072323A2030782530386C78AE
:105A00000A20202072333A2030782530386C780A0A
:105A10000020207231323A2030782530386C780AF4
:105A20002020206C723A2030782530386C780A209B
:105A3000202070633A2030782530386C780A202096
:105A40007073723A2030782530386C780A0A004634
:105A500053522F4641523A0020434653523A203087
:105A6000782530386C780A0020484653523A203066
:105A7000782530386C780A0020444653523A20305A
:105A8000782530386C780A0020414653523A20304D
:105A9000782530386C780A0020424641523A20304E
:105AA000782530386C780A004D4D4641523A203006
:105AB000782530386C780A004D6973630045584387
:105AC0005F5245543A2030782530386C780A0041CE
:105AD0007474656D7074696E6720746F207265638D
:105AE0006F6E73747275637420737461746520666D
:105AF0006F7220646562756767696E672E2E2E006F
:105B0000496E204744423A0A20207365742024706D
:105B1000633D3078256C780A20206672616D6520BF
:105B2000300A202062740A000A49535220737461BB
:105B3000636B206F766572666C6F7765642062793F
:105B4000206174206C65617374202564206279740F
:105B500065732E0A0048415244204641554C54205A
:105B600048414E444C4552004D454D204D414E411B
:105B700047452048414E444C4552004E4D4920482F
:105B8000414E444C455200555341474520464155EE
:105B90004C542048414E444C4552004641494C45E6
:105BA0004420415353455254494F4E2E0025700A0C
:105BB000002A2A2A2052494F54206B65726E656C68
:105BC0002070616E69633A0A25730A0A002A2A2A3C
:105BD0002068616C7465642E0A0A006D61696E2824
:105BE000293A20546869732069732052494F54211F
:105BF000202856657273696F6E3A20323031372E25
:105C000030312D646576656C2D3235352D67316602
:105C10006232312D56616E64726973290A006964BB
:105C20006C65006D61696E00496E73696465206919
:105C300073722025640A0000004400400000020046
:105C40000300024002000240070026060400000094
:105C50000048004000000400090C0240080C02400B
:105C600007002703040000005F517374617465002E
:105C70006E616D650009706964207C20252D3231CC
:105C8000737C20252D397351207C20707269207C13
:105C900020737461636B2028207573656429207CF0
:105CA0002062617365202020202020207C206375E5
:105CB0007272656E74202020200A000920202D2099
:105CC0007C206973725F737461636B2020202020D5
:105CD000202020202020207C202D2020202020205B
:105CE00020202D207C2020202D207C20253569207F
:105CF0002825356929207C2025313070207C2025FD
:105D00003130700A000925336869207C20252D3246
:105D10003073207C20252D387320252E3173207C74
:105D200020253369207C20253569202825356929DF
:105D3000207C2025313070207C2025313070200AD5
:105D4000007C0053554D000925357320252D323137
:105D5000737C25313373253673202535692028253A
:105D60003569290A0073746F7070656400736C651F
:105D70006570696E6700626C206D7574657800628D
:105D80006C20727800626C2073656E6400626C2017
:105D90007265706C7900626C20616E79666C00626D
:105DA0006C20616C6C666C0072756E6E696E67005B
:105DB00070656E64696E6700676E72635F6E6574AE
:105DC000646576323A20706F737369626C79206C07
:105DD0006F737420696E746572727570742E0055DD
:105DE0006E6578706563746564206576656E742091
:105DF000726563656976656400756E657870656364
:105E0000746564206D65737361676520747970656E
:105E10000000000000030000060C024002100240D7
:105E2000070C02400A0C0240415438365246327880
:105E3000782064657669636520647269766572208E
:105E40007465737400496E697469616C697A696E0E
:105E5000672041543836524632787820726164693E
:105E60006F206174205350495F2564200A007265D9
:105E700063765F746872656164004372656174691A
:105E80006F6E206F66207265636569766572207437
:105E90006872656164206661696C656400496E6959
:105EA0007469616C697A6174696F6E20737563637C
:105EB00065737366756C202D207374617274696EDE
:105EC0006720746865207368656C6C206E6F77005E
:105ED000F45E0008FD5E0008B11B00080F5F0008BB
:105EE000165F0008BD1B0008000000000000000055
:105EF000000000006966636F6E66696700436F6E3D
:105F0000666967757265206E6574646576320074C3
:105F10007874736E640053656E642049454545206E
:105F20003830322E31352E34207061636B65740049
:105F300049666163652025336420204857616464A5
:105F4000723A20002C204C6F6E67204857616464C1
:105F5000723A20002C2050414E3A203078253034BF
:105F600078002865727229000A2020202020202035
:105F70002020202041646472657373206C656E6715
:105F800074683A202575002C20536F757263652064
:105F900061646472657373206C656E6774683A201F
:105FA0002575002C204D61782E5061796C6F6164ED
:105FB0003A202575000A20202020202020202020A3
:105FC0002049507636204949443A20000A202020B2
:105FD00020202020202020204368616E6E656C3ACE
:105FE000202575002C2043682E706167653A2025B6
:105FF00075002C205458506F7765723A2025642024
:1060000064426D002C20776972656C657373002C97
:106010002077697265640020202020202020202025
:106020000020205052454C4F4144002020415554FF
:106030004F41434B002020524157002020415554EE
:106040004F43434100202043534D41007573616726
:10605000653A202573203C69666163653E205B3CA0
:1060600070616E3E5D203C616464723E203C7465EC
:1060700078743E0A00747874736E643A2025642044
:106080006973206E6F7420616E20696E746572662C
:106090006163650A00747874736E643A20457272A5
:1060A0006F72207072657065726172696E672066CA
:1060B00072616D6500747874736E643A2045727213
:1060C0006F72206F6E2073656E64696E67007478FE
:1060D00074736E643A2073656E642025752062794E
:1060E00074657320746F2000202850414E3A2000C0
:1060F000556E6578706563746564204D48522066FE
:106100006F7220696E636F6D696E67207061636B7B
:10611000657400424541434F4E0044415441004D97
:106120004143434D4400554E4B4E4F574E0044653E
:1061300073742E2050414E3A203078253034782C1C
:1061400020446573742E20616464722E3A20000A24
:106150005372632E2050414E3A20307825303478E7
:106160002C205372632E20616464722E3A20000A40
:1061700053656375726974793A2000312C200030C0
:106180002C20004672616D652070656E642E3A2089
:106190000041434B207265712E3A200050414E2041
:1061A000636F6D702E3A2000310056657273696F0F
:1061B0006E3A200025752C20005365712E3A20255B
:1061C000750A007478743A20000A202020202000EC
:1061D000525353493A2025752C204C51493A2025D9
:1061E000750A0A000102030402020202020204000C
:1061F0001327000899260008352600088125000885
:1062000081270008212300080F0F0F0E0E0E0E0D20
:106210000D0C0C0B0B0A0908070605030000030010
:10622000030002000200010001000000FFFFFEFF6A
:10623000FDFFFCFFFBFFF9FFF7FFF4FFEFFFFFFFA0
:106240002530396F0025303678002530376400203E
:1062500020202025630020253036686F002025305F
:1062600031326C6F0020253032346C6C6F00202589
:10627000253025646F002025253025646C6F0020B3
:1062800025346400202536686400202531326C6492
:1062900000202532346C6C640020252525646400C0
:1062A00020252525646C64002025337500202536C3
:1062B000687500202531326C7500202532346C6CF5
:1062C00075002025252575750020252525756C75FB
:1062D00000202530327800202530346878002025D1
:1062E00030386C780020253031366C6C78002025F1
:1062F0002530257578002025253025756C780020FF
:1063000020205C30002020205C61002020205C6286
:10631000002020205C66002020205C6E00202020D1
:106320005C72002020205C74002020205C7600201D
:10633000202530336F0025730001007368656C6C95
:106340003A20696E636F72726563742071756F7441
:10635000696E670068656C7000446573637269708C
:1063600074696F6E00436F6D6D616E6400252D3230
:1063700030732025730A002D2D2D2D2D2D2D2D2D23
:106380002D2D2D2D2D2D2D2D2D2D2D2D2D2D2D2D3D
:106390002D2D2D2D2D2D2D2D2D2D2D2D2D2D007314
:1063A00068656C6C3A20636F6D6D616E64206E6F12
:1063B0007420666F756E643A2025730A0000000031
:1063C000E4630008EB6300088D3D0008FB630008F0
:1063D000FE630008973D0008000000000000000078
:1063E000000000007265626F6F74005265626F6F2B
:1063F0007420746865206E6F64650070730050725D
:10640000696E747320696E666F726D6174696F6E08
:106410002061626F75742072756E6E696E6720748C
:106420006872656164732E000000000000000000C7
:10643000000000000000000000000000000000005C
:10644000000000000000000000000000000000004C
:10645000000000000000000000000000000000003C
:10646000000000000000000000000000000000002C
:10647000000000000000000000000000000000001C
:106480000000000000000000540200204300504FB4
:1064900053495800232D302B2000686C4C00656652
:1064A0006745464700303132333435363738394165
:1064B000424344454600303132333435363738397B
:1064C0006162636465660000202020202020202077
:1064D0002028282828282020202020202020202094
:1064E00020202020202020208810101010101010B4
:1064F00010101010101010100404040404040404FC
:10650000040410101010101010414141414141018C
:10651000010101010101010101010101010101016B
:10652000010101101010101010424242424242027A
:10653000020202020202020202020202020202023B
:1065400002020210101010200000000000000000E5
:10655000000000000000000000000000000000003B
:10656000000000000000000000000000000000002B
:10657000000000000000000000000000000000001B
:10658000000000000000000000000000000000000B
:1065900000000000000000000000000000000000FB
:1065A00000000000000000000000000000000000EB
:1065B00000000000000000000000000000000000DB
:0865C0000000000000000000D3
:1065C800D813002000000000F8040020400000005C
:1065D80000000000000000001E5C0008235C0008AA
:1065E800FF000000655D00086D5D0008765D00082D
:1065F8007F5D0008855D00088D5D0008965D0008D8
:106608009F5D000800000000A85D0008B05D00085C
:106618005402002000000000486400086864000874
:1066280028640008000000000000000000000000CE
:106638000000000000000000000000000000000052
:106648000000000000000000000000000000000042
:106658000000000000000000000000000000000032
:106668000000000000000000000000000000000022
:1066780000000000430000000000000000000000CF
:106688000000000000000000000000000000000002
:1066980000000000430000000000000000000000AF
:1066A80000000000000000000000000000000000E2
:1066B800000000004300000000000000000000008F
:1066C80000000000000000000000000000000000C2
:1066D800000000004300000000000000000000006F
:1066E80000000000000000000000000000000000A2
:1066F800000000004300000000000000000000004F
:106708000000000000000000000000000000000081
:10671800000000004300000000000000000000002E
:106728000000000000000000000000000000000061
:10673800000000004300000000000000000000000E
:106748000000000000000000000000000000000041
:1067580000000000ED570008554E0008000000003A
:10676800C7640008FE5A0008DA5B0008DA5B000814
:10677800DA5B0008DA5B0008DA5B0008DA5B00081D
:10678800DA5B0008DA5B0008DA5B0008FFFFFFFF4E
:10679800FFFFFFFFFFFFFFFFFFFF00000100415366
:1067A800434949000000000000000000000000000C
:1067B800000000000000000000000000000041533D
:1067C80043494900000000000000000000000000EC
:1067D80000000000000000000000000000000000B1
:04000005080004A546
:00000001FF
